:04000000CAEF08F04B
:1000080000C019F001C018F002C017F003C016F0C4
:1000180004C015F09EA002D09E9091DB9EA203D052
:100028009E9232EC06F019C000F018C001F017C01B
:0C00380002F016C003F015C004F0110027
:10004400220E0C6E086A096A0A6A0B6A0C06D8B496
:100054001FD0D8900B320A320932083203320232EE
:1000640001320032D8A0F2D70C06D8B409D004501B
:1000740008260550092206500A2207500B22EAD707
:10008400045008260550092206500A2207500B2264
:02009400120058
:10009600000E006E7D0E016E000E026E036E1200E3
:1000A6000B6A0A6A096A086A0E6A0334083604503B
:1000B600085E0550D8A0053C095E0650D8A0063C4F
:1000C6000A5E0750D8A0073C0B5EE86AD8A0010E6E
:1000D6000E5E0336070E0C6E0334083609360A36F2
:1000E6000B360E36045003A012D0085E0550D8A079
:1000F600053C095E0650D8A0063C0A5E0750D8A00B
:10010600073C0B5EE86AD8A0010E0E5E11D00826E9
:100116000550D8B0053C09260650D8B0063C0A263C
:100126000750D8B0073C0B26E86AD8B0010E0E2659
:1001360003360C2ED1D70234083609360A360B366A
:100146000E36045003A012D0085E0550D8A0053C18
:10015600095E0650D8A0063C0A5E0750D8A0073CA8
:100166000B5EE86AD8A0010E0E5E11D00826055077
:10017600D8B0053C09260650D8B0063C0A260750DA
:10018600D8B0073C0B26E86AD8B0010E0E26023618
:10019600070E0C6E0234083609360A360B360E3652
:1001A600045002A012D0085E0550D8A0053C095E96
:1001B6000650D8A0063C0A5E0750D8A0073C0B5E46
:1001C600E86AD8A0010E0E5E11D008260550D8B0F8
:1001D600053C09260650D8B0063C0A260750D8B07A
:1001E600073C0B26E86AD8B0010E0E2602360C2E06
:1001F600D1D70134083609360A360B360E36045086
:1002060002A012D0085E0550D8A0053C095E065033
:10021600D8A0063C0A5E0750D8A0073C0B5EE86AE9
:10022600D8A0010E0E5E11D008260550D8B0053CA8
:1002360009260650D8B0063C0A260750D8B0073C17
:100246000B26E86AD8B0010E0E260136070E0C6E94
:100256000134083609360A360B360E36045001A02C
:1002660012D0085E0550D8A0053C095E0650D8A0FD
:10027600063C0A5E0750D8A0073C0B5EE86AD8A089
:10028600010E0E5E11D008260550D8B0053C092691
:100296000650D8B0063C0A260750D8B0073C0B26B5
:1002A600E86AD8B0010E0E2601360C2ED1D70034DE
:1002B600083609360A360B360E36045001A012D01F
:1002C600085E0550D8A0053C095E0650D8A0063C3D
:1002D6000A5E0750D8A0073C0B5EE86AD8A0010E5C
:1002E6000E5E11D008260550D8B0053C09260650EA
:1002F600D8B0063C0A260750D8B0073C0B26E86A59
:10030600D8B0010E0E260036070E0C6E00340836E5
:1003160009360A360B360E36045000A012D0085E97
:100326000550D8A0053C095E0650D8A0063C0A5EDA
:100336000750D8A0073C0B5EE86AD8A0010E0E5EF7
:1003460011D008260550D8B0053C09260650D8B06D
:10035600063C0A260750D8B0073C0B26E86AD8B0F8
:10036600010E0E2600360C2ED1D700B00ED004504A
:1003760008260550D8B0053C09260650D8B0063CDC
:0C0386000A260750D8B0073C0B261200D6
:100392005F065F065FC001F05F060150000803E2DE
:1003A20000000000F7D7000000000000000000007D
:0203B200120037
:1003B400086A096A100E0C6E0134083609360450B6
:1003C400085E0550D8A0053C095ED8B007D004509B
:1003D40008260550D8B0053C0926D89000360136C9
:0603E4000C2EEAD7120006
:1003EA0055DEE80E046E030E056E000E066E076EED
:1003FA0024DE00C05BF001C05CF002C05DF003C007
:10040A005EF053C004F054C005F0000E066E076E8D
:10041A0045DE00C05BF001C05CF002C05DF003C0C5
:10042A005EF000C005F001C006F002C007F003C08C
:10043A0008F00832073206320532089E08320732BF
:10044A0006320532089E05C000F006C001F007C05A
:10045A0002F008C003F00332023201320032039E76
:10046A0000C057F001C058F011DE55C004F056C064
:10047A0005F0000E066E076EE0DD57C009F058C0A1
:10048A000AF0000E0B6E0C6E030E086E09C004F023
:10049A000AC005F00BC006F00CC007F0085007E0D0
:1004AA0004360490053606360736FF0FF8D7F6DD10
:1004BA0000C05BF001C05CF002C05DF003C05EF0FA
:1004CA000A0E046E000E056E57C000F058C001F007
:1004DA006CDF00C057F001C058F0000E015C02E169
:1004EA00030E005C01E241D04CC0E9FF4DC0EAFFB7
:1004FA005E50000808E15D50000805E15C50000804
:10050A0002E15B5000082FE24B50EF1258520DE007
:10051A00596A5A6A000E5A5C02E15850595C05E25F
:10052A005F6A32DF594A5A2AF5D757C05FF02CDF83
:10053A004A50EF1658520DE0596A5A6A000E5A5C30
:10054A0002E15850595C05E25F6A1EDF594A5A2A8D
:10055A00F5D757C05FF018DF010E5B5E000E5C5ADC
:0C056A005D5A5E5AC5D74A50EF161200C9
:100576004F904FB002D04E9A01D04E8A4EBA02D05A
:100586004E9801D04E884EB802D04E9E01D04E8E67
:100596004EBE02D04E9C01D04E8C4E904EB002D034
:1005A6004E9401D04E844EB402D04E9201D04E826B
:1005B6004EB202D04E9601D04E864EB602D04F9421
:1005C60001D04F844FB402D04F9201D04F824FB228
:1005D60002D04F9801D04F884FB802D04F9601D025
:1005E6004F86436A446A326A306A316A356A366AC5
:1005F600336A346A2E6A2F6A2C6A2D6A396A406A0F
:10060600466A476A486A426A416A456A3D6A3C6A7E
:100616003F6A3E6A3B6A386A376A3A6A246A236ADC
:10062600226A256A286A276A266A2B6A899E89BEF3
:1006360002D0899C01D0898C89BC02D0899A01D0CC
:10064600898A89BA02D0899801D0898889B802D066
:10065600899601D0898689B602D0899401D0898489
:1006660089B402D0899201D0898289B202D0899058
:1006760001D089808C988CB802D08C9A01D08C8A53
:100686008CBA02D08C9C01D08C8C8CBC02D08C9EF7
:1006960001D08C8E8CBE02D08B9001D08B808BB01B
:1006A60002D08B9201D08B828BB202D08C9201D079
:1006B6008C828CB202D08C9001D08C801D6A1C6A10
:1006C6001B6A1E6A216A206A1F6A1A6A8D908B8AC3
:1006D6008BBA02D08B9601D08B868BB602D08D92C8
:1006E60001D08D828B988BB802D08B9401D08B84ED
:1006F6008BB402D08D9401D08D848B9E8A988A9A71
:020706001200DF
:080708000C0ECA6E9D82120066
:08071000B10ECD6E9D801200B8
:10071800700ED36E9B8C0F0EC16E070EB46E27DF62
:10072800926ACF0E936E400E946E080E956E969058
:0E07380096929694E5DFE8DFF28EF28C1200C6
:10074600D80ECF6EF00ECE6E81B24F804FB009D06C
:1007560081A007D08AA805D0040E295C02E2292AC6
:1007660007DF2950040A02E18AB84F804FB08A8A0F
:1007760081B603D08D828D9402D08D928D8482BCF9
:1007860003D08B868B9402D08B968B8481BC03D04E
:100796008B8A8B9802D08B9A8B884FA052D081ACD3
:1007A6004BD0434A442A000E006E4450005C02E1DE
:1007B6004350500802E21D6A8A88000E006E4450BB
:1007C600005C02E143504608D8A01C6A000E006E89
:1007D6004450005C02E143503C08D8A01B6A000E5E
:1007E600006E4450005C02E143503208D8A01E6AF5
:1007F600000E006E4450005C02E143502808D8A069
:10080600216A000E006E4450005C02E143501E084F
:10081600D8A0206A000E006E4450005C02E14350EE
:100826001408D8A01F6A000E006E4450005C02E156
:1008360043500A08D8A01A6A83A603D099DE296A0B
:100846000DD281AEA7D08B8E81BC03D083A401D0FC
:1008560001D04E8C82BC08D02F50020802E12E50E7
:10086600EE0802E2354A362A000E2F1802E1000E83
:100876002E18D8B48ED02F50020802E12E50EE0862
:1008860045E2030E1F6E030E1C6E4F984E84EE0E4D
:100896002E5C036E020E2F58046E03C000F004C0D7
:1008A60001F001320032019E01320032019E00C089
:1008B60026F000C023F0304A312A000E006E315077
:1008C600005C02E13050FA0820E2010E315C02E1E0
:1008D600F40E305C1AE2030E1A6E030E1D6E4F966E
:1008E6004E80FA0E305C036E000E3158046E03C063
:1008F60000F004C001F001320032019E01320032E4
:10090600019E00C02BF000C024F043D02F500108F8
:1009160002E12E50F4081BE2030E206E030E1B6E3E
:100926004F924E82F40E2E5C036E010E2F58046E0B
:1009360003C000F004C001F001320032019E013212
:100946000032019E00C027F000C022F022D0000E27
:10095600006E2F50005C02E12E50FA081AE2030ED8
:10096600216E030E1E6E4F944E86FA0E2E5C036E9B
:10097600000E2F58046E03C000F004C001F00132CF
:100986000032019E01320032019E00C028F000C0F4
:1009960025F001D08B9E81AC73D04FB071D081BE53
:1009A6004E8C3650020802E13550580807E3010E16
:1009B600365C02E1900E355C01E301D04E8C33C00B
:1009C60001F034C002F0334A342A000E006E0250A1
:1009D600005C02E10150460809E21A6A1F6A206AB1
:1009E600216A1E6A1B6A1C6A8A884AD0000E006E3B
:1009F6003450005C02E133503C0807E21A6A1F6A71
:100A0600206A216A1E6A1B6A3BD0000E006E3450B3
:100A1600005C02E13350320806E21A6A1F6A206A55
:100A2600216A1E6A2DD0000E006E3450005C02E171
:100A36003350280805E21A6A1F6A206A216A20D004
:100A4600000E006E3450005C02E133501E0804E2D2
:100A56001A6A1F6A206A14D0000E006E3450005CB9
:100A660002E13350140803E21A6A1F6A09D0000E25
:100A7600006E3450005C02E133500A08D8A01A6AAE
:100A86008AA80BD081AC09D04FB007D032C001F094
:100A9600322A01503208D8A04E8C81A670D081BC73
:100AA60005D081AE03D083A401D001D04E8C2C4A50
:100AB6002D2A2D50020802E12C502608D8A04E8C73
:100AC600000E2D5C02E17D0E2C5C0FE2010E1D6E08
:100AD6002CC000F02DC001F001320032019E01321F
:100AE6000032019E00C03DF04AD0000E2D5C02E1AE
:100AF600FA0E2C5C15E2010E1C6E7D0E2C5C036E4C
:100B0600000E2D58046E03C000F004C001F001323F
:100B16000032019E01320032019E00C03CF02FD00F
:100B2600010E2D5C02E1770E2C5C15E2010E1B6EA8
:100B3600FA0E2C5C036E000E2D58046E03C000F0F6
:100B460004C001F001320032019E01320032019EE2
:100B560000C03FF014D0010E1E6E770E2C5C036EA3
:100B6600010E2D58046E03C000F004C001F00132DE
:100B76000032019E01320032019E00C03EF082AC7E
:100B86006DD02E4A2F2A000E2F5C02E1FA0E2E5C43
:100B960012E2020E216E2EC000F02FC001F00132CB
:100BA6000032019E01320032019E01320032019E66
:100BB60000C048F053D0010E2F5C02E1F40E2E5C0B
:100BC60018E2020E206EFA0E2E5C036E000E2F58EF
:100BD600046E03C000F004C001F001320032019E31
:100BE60001320032019E01320032019E00C042F005
:100BF60035D0020E2F5C02E1EE0E2E5C18E2020EDC
:100C06001F6EF40E2E5C036E010E2F58046E03C089
:100C160000F004C001F001320032019E01320032C0
:100C2600019E01320032019E00C041F017D0020E33
:100C36001A6EEE0E2E5C036E020E2F58046E03C063
:100C460000F004C001F001320032019E0132003290
:0E0C5600019E01320032019E00C045F01200E6
:100C64002AC001F02A2A01507E0AD8B42A6A3CD04C
:100C74008C908CB002D0899001D0898042D08C9025
:100C84003A502A5C02E2898001D089903AD0899056
:100C940045502A5C02E28C8001D08C9032D0497E8F
:100CA40049AE07D08C908CB002D0899001D0898055
:100CB40028D04FB609D02B502A5C03E289808C904F
:100CC40002D089908C8008D02B502A5C03E2899052
:100CD4008C8002D089808C9014D08C908CB002D0FF
:100CE400899001D089800DD01A50000AC1E01A50B1
:100CF400010AC5E01A50020ACAE01A50030ACFE0FA
:100D0400ECD73CD08C928CB202D0899201D08982EB
:100D140042D08C9237502A5C02E2898201D08992B7
:100D24003AD0899241502A5C02E28C8201D08C92A2
:100D340032D0497C49AC07D08C928CB202D08992D3
:100D440001D0898228D04FB809D026502A5C03E20A
:100D540089828C9202D089928C8208D026502A5C97
:100D640003E289928C8202D089828C9214D08C9274
:100D74008CB202D0899201D089820DD01F50000A12
:100D8400C1E01F50010AC5E01F50020ACAE01F500B
:100D9400030ACFE0ECD73CD08B928BB202D089947B
:100DA40001D0898442D08B9238502A5C02E2898433
:100DB40001D089943AD0899442502A5C02E28B8211
:100DC40001D08B9232D0497649A607D08B928BB250
:100DD40002D0899401D0898428D04FB209D02750F9
:100DE4002A5C03E289848B9202D089948B8208D096
:100DF40027502A5C03E289948B8202D089848B92E7
:100E040014D08B928BB202D0899401D089840DD0F6
:100E14002050000AC1E02050010AC5E02050020A17
:100E2400CAE02050030ACFE0ECD73CD08B908BB0C3
:100E340002D0899601D0898642D08B903B502A5C9F
:100E440002E2898601D089963AD0899648502A5C74
:100E540002E28B8001D08B9032D0497849A807D028
:100E64008B908BB002D0899601D0898628D04FB45C
:100E740009D028502A5C03E289868B9002D0899697
:100E84008B8008D028502A5C03E289968B8002D09C
:100E940089868B9014D08B908BB002D0899601D028
:100EA40089860DD02150000AC1E02150010AC5E015
:100EB4002150020ACAE02150030ACFE0ECD73CD00B
:100EC4008C9E8CBE02D0899801D0898842D08C9E99
:100ED4003E502A5C02E2898801D089983AD08998E8
:100EE40047502A5C02E28C8E01D08C9E32D0497A23
:100EF40049AA07D08C9E8CBE02D0899801D08988DB
:100F040028D04EB609D025502A5C03E289888C9EED
:100F140002D089988C8E08D025502A5C03E28998E7
:100F24008C8E02D089888C9E14D08C9E8CBE02D06C
:100F3400899801D089880DD01E50000AC1E01E5046
:100F4400010AC5E01E50020ACAE01E50030ACFE09F
:100F5400ECD73CD08C9C8CBC02D0899A01D0898A75
:100F640042D08C9C3F502A5C02E2898A01D0899A43
:100F74003AD0899A46502A5C02E28C8C01D08C9C2F
:100F840032D0497449A407D08C9C8CBC02D0899A75
:100F940001D0898A28D04EB209D022502A5C03E2BB
:100FA400898A8C9C02D0899A8C8C08D022502A5C25
:100FB40003E2899A8C8C02D0898A8C9C14D08C9CF4
:100FC4008CBC02D0899A01D0898A0DD01B50000AAA
:100FD400C1E01B50010AC5E01B50020ACAE01B50C5
:100FE400030ACFE0ECD73CD08C9A8CBA02D0899C0F
:100FF40001D0898C42D08C9A3C502A5C02E2898CC4
:1010040001D0899C3AD0899C40502A5C02E28C8AA7
:1010140001D08C9A32D0497049A007D08C9A8CBAEE
:1010240002D0899C01D0898C28D04EB409D0235099
:101034002A5C03E2898C8C9A02D0899C8C8A08D021
:1010440023502A5C03E2899C8C8A02D0898C8C9A76
:1010540014D08C9A8CBA02D0899C01D0898C0DD082
:101064001C50000AC1E01C50010AC5E01C50020AD1
:10107400CAE01C50030ACFE0ECD73CD08C988CB863
:1010840002D0899E01D0898E42D08C983D502A5C32
:1010940002E2898E01D0899E3AD0899E39502A5C19
:1010A40002E28C8801D08C9832D0497249A207D0D0
:1010B4008C988CB802D0899E01D0898E28D04EB0ED
:1010C40009D024502A5C03E2898E8C9802D0899E30
:1010D4008C8808D024502A5C03E2899E8C8802D034
:1010E400898E8C9814D08C988CB802D0899E01D0AB
:1010F400898E0DD01D50000AC1E01D50010AC5E0C3
:101104001D50020ACAE01D50030ACFE0ECD71200BA
:1011140050C04CF051C04DF052C001F0010E006EB1
:10112400015004E000360090FF0FFBD700C04BF0E5
:10113400001E00C04AF0120E5024E96E000E512029
:10114400EA6E0050EF16120EE95E0050EF16120020
:10115400EE0E506E020E516E030E515C02E1070E4C
:10116400505C0DE250C053F051C054F0190E556E4E
:10117400000E566EF5EC01F0504A512AEDD71200DC
:101184000900F5CFE6FF0006FBE10106F9E11200D4
:10119400F2EC08F08CEC03F08D0E506E0F0E516ED5
:1011A400526AB6DF4EAC02D0D3DF4E9CFBD7FFD7DA
:1011E40010EE1AF02F0E006E010E016EB40EF66EA4
:0E11F400110EF76E000EF86EC2EC08F012003D
:0111B400003A
:0111B5000039
:0111B6000038
:0111B7000037
:0111B8000036
:0111B9000035
:0111BA000034
:0111BB000033
:0111BC000032
:0111BD000031
:0111BE000030
:0111BF00002F
:0111C000002E
:0111C100002D
:0111C200002C
:0111C300002B
:0111C400002A
:0111C5000029
:0211C600000027
:0211C800000025
:0211CA00000023
:0111CC000022
:0211CD00000020
:0211CF0000001E
:0111D100001D
:0111D200001C
:0111D300001B
:0111D400001A
:0111D5000019
:0111D6000018
:0111D7000017
:0111D8000016
:0111D9000015
:0111DA000014
:0111DB000013
:0111DC000012
:0211DD00000010
:0111DF00000F
:0111E000000E
:0111E100000D
:0111E200000C
:020000040030CA
:0D000100081E1EFF8181FF0FC00FE00F40A1
:00000001FF
